:03000000022E28A5
:0C2E280078FFE4F6D8FD758175022E6F6E
:100FA90020000A3C2E2E2E3E004950436F6E6E657E
:100FB90063745245510A004950436F6E6E656374FC
:100FC900000A49504E6F41434B210A003E432C56BB
:100FD9002C43432CC0E4E0EFF2E5F020D1E8EDEA40
:100FE900EEEC49500A003E432C4D41432C2530324A
:100FF90062583A25303262583A25303262583A25D9
:10100900303262583A25303262583A2530326258C5
:101019002C4D414320E0E4F0E5F10A003E432C5613
:1010290045522C20332E3220EEF2202573202573D1
:101039002CC2E5F0F1E8FF20495020ECEEE4F3EB97
:10104900FF0A0041756720303720323031320031D4
:10105900353A33363A3432003E432C4C442C505204
:101069004F473A2020202020202020202020202007
:101079002020202020202020202020202020202067
:101089002020202020202020202020202020202057
:101099002020202020202020202020202020202047
:1010A90020202020202020202CC4E0F2E020EFF096
:1010B900EEF8E8E2EAE828F4E0E9EB290A003E2A3A
:1010C9002C312CCEF1EDEEE2EDFBE520EFE0F0E086
:1010D900ECE5F2F0FB20F1E5F2E5E2EEE3EE20E8E3
:1010E900EDF2E5F0F4E5E9F1E00A003E412C41308A
:1010F900312C2562752E2562752E2562752E256285
:10110900752C495020E0E4F0E5F120E0E4E0EFF24D
:10111900E5F0E00A003E412C4130322C2562752E63
:101129002562752E2562752E2562752C495020E0A1
:10113900E4F0E5F120EEF1ED2E20F1E5F0E2E5F045
:10114900E00A003E412C4130332C2562752E256280
:10115900752E2562752E2562752C495020E0E4F024
:10116900E5F120F0E5E72E20F1E5F0E2E5F0E00A0F
:10117900003E412C4130342C2562752E2562752E96
:101189002562752E2562752CCCE0F1EAE020F1E5A7
:10119900F2E80A003E412C4130352C2562752E2596
:1011A90062752E2562752E2562752CD8EBFEE70A2D
:1011B900003E2A2C312CC4EEEF2E20EFE0F0E0ECBB
:1011C900E5F2F0FB20F1E5F2E5E2EEE3EE20E8EDF1
:1011D900F2E5F0F4E5E9F1E00A003E422C53303142
:1011E9002C2562752CC6E4E0F2FC20E7E0EFF0EE76
:1011F900F1E020F1EEE5E4E8EDE5EDE8FF20EEF2BF
:1012090020F1E5F0E2E5F0E00A003E422C533032ED
:101219002C2562752CCEE1ECE5ED20F120F1E5F00D
:10122900E2E5F0EEEC20E1E5E720EAE2E8F2E0EDC4
:10123900F6E8E90A003E422C5330332C2562752C1E
:10124900CFE5F0E5E7E0EFF3F1EA20EFF0E820EF92
:10125900EEF2E5F0E520F1E2FFE7E820F120F1E523
:10126900F0E2E5F0EEEC0A003E422C5330382C2532
:1012790062752CCCE5E4EBE5EDEDFBE92049502066
:10128900EAE0EDE0EB28E7E0E4E5F0E6EAE020E477
:10129900EE203520F1E5EA290A003E422C5330358B
:1012A9002C2562752CCAE0EDE0EB20F8E8F0EEEAB7
:1012B900EEE2E5F8E0F2E5EBFCEDEEE3EE20EEE13F
:1012C900ECE5EDE00A003E532C5330362C25303244
:1012D90062582530326258253032625825303262E0
:1012E90058253032625825303262582C4D414320FE
:1012F900E0E4F0E5F120F8E8F0EEEAEEE2E5F8E006
:10130900F2E5EBFCEDEEE3EE20EEE1ECE5EDE00AD3
:10131900003E454E440A000A44756D70582020204D
:10132900202030302030312030322030332030340A
:1013390020303520303620303720303820303920E1
:101349003041203042203043203044203045203085
:1013590046000A3A003A20000A000A44756D7044B2
:1013690020202020203030203031203032203033EE
:1013790020303420303520303620303720303820A6
:101389003039203041203042203043203044203051
:101399004520304600457272206B65790052642001
:1013A900656570726F6D0A005264204D454D0A00E3
:1013B900526420436F64650A00577269746520435B
:1013C9006F64650A0044656275674950204F4E0A8B
:1013D9000044656275674950204F46460A004465D6
:1013E90062756755736572204F6E0A0044656275B0
:1013F9006755736572204F46460A004465627567F2
:101409004D7367204F6E0A0044656275674D7367B7
:10141900204F46460A00436F6E666967206C6F630A
:101429006B210A00577220656570726F6D0A002082
:101439005361766520656570726F6D210A0045728A
:1014490072204D414321004C6F61643E3E002A00E9
:10145900CEF8E8E1EAE00A00202D20257528257557
:10146900290A003C4130313D003C4130323D003CCD
:101479004130333D003C4130343D003C4130353D45
:10148900003C21003C5330313D003C5330323D009B
:101499003C5330333D003C5330353D003C533038EC
:0814A9003D003C5330363D00CC
:0636250001130001110079
:10367500C28E438910E4F58B758DB8D2ABD28E22FC
:03001B00022D981B
:102D9800C0E0C083C082C0D0C28E758B00758DB86C
:102DA800201C0675A61E75A6E10511D218E513604C
:102DB8000205130516E516540F7051E512D3940158
:102DC80040021512D224E516543F7012D2169066AE
:102DD8008EE0600A04F0E0D394B44002D21C9066FE
:102DE80087E0600204F0906104E0600214F09066ED
:102DF8008FE0D394014003E014F0301B020514E582
:102E080015D394644004D21C80020515E510D394B0
:102E18000140021510D28ED0D0D082D083D0E032BB
:10092100C291C290D2B5C2217D027C007F071236EE
:10093100088F26E526646060097D017F601235A37A
:10094100D221E4FDFC7F0B1236088F26E52630E626
:10095100097D04E4FF1235C7D2217D017C007F07A8
:100961001236088F26E5267008FD7FFF1235A3D2C7
:1009710021302103126000C288C2A8C2AA75890071
:1009810012315090633FE0B4FA06A3E064CE607B7D
:10099100E4F52674372526F582E43463F583E4F023
:1009A1000526E526B443EC90633F74FAF0A374CEB8
:1009B100F0A374CCF0906345740AF0E4A3F0A304AF
:1009C100F0A3F090633B74FFF0A3F0A3F0E4A3F075
:1009D1009063567403F0E4F526E5262401FFE43321
:1009E100FE74372526F582E43463F583E0FD123584
:1009F1007F0526E526C3944340DFE4F5A775A61ECF
:100A010075A6E1907FF0F0A3F080FE90634A740335
:100A1100F0A374CCF0E4906349F090668CF0A3F0FD
:100A21001228EFC2B512365BC21C1233CDD221C2DD
:100A310023C2229065777408F09062B57424F0E4C3
:100A4100A3F090633FE09062B7F0906340E0906262
:100A5100B8F0906341E09062B9F0906342E0906237
:100A6100BAF0906343E09062BBF0906344E090621F
:100A7100BCF0751201E4906578F0C21DC21EC21F60
:100A8100C220202118AF26FE7D031229D5E4FF12D2
:100A91002C467E0F7FA9E4FBFDFC1225FC90668E9F
:100AA100E060037401F0E4906104F0F51490657660
:100AB100F0F51512367575A70775A61E75A6E1D254
:100AC100AFE4F515906104E0700312210390668F85
:100AD100E06401701D9080007410F09080A874FF94
:100AE100F0A3F0A3F0A3F0E490668FF0D221C2222C
:100AF100C223908008E0F52630E405D21D7410F081
:100B0100E52630E508D21F9080087420F0E52630F4
:100B1100E608D21E9080087440F0E514C3940340A7
:100B210019908002E4F0908001F0908000F0E514CB
:100B310094064006E4F5141233CD9080A0E07003D2
:100B41001232489080B8E070031231CE9080D0E02C
:100B51007003123371908000E07013301D10122762
:100B610003906332EFF0D39400400312003690807B
:100B710002E07006908000E06005D21B020AC2C24A
:100B81001BE4F514906104E06003020AC220211203
:100B9100906579E0600C7E0F7FAB122807E49065C9
:100BA10079F0301F12121F92906332EFF0D394004C
:100BB1004005E0FF120032201E03020D46121E0BFB
:100BC100906332EFF07003020AC2906376E054BF83
:100BD100247F7003020CA1147003020C79240260BB
:100BE10003020CE82021077E0F7FB212280720257F
:100BF10003020D4690634EE07006906352E0606719
:100C0100906683E0FF90634EE0B50724906684E030
:100C1100FE90634FE0B50618906685E0FE90635044
:100C2100E0B5060C906686E0FE906351E06E603799
:100C3100906352E06F6003020D46906684E0FF907E
:100C41006353E06F6003020D46906685E0FF906399
:100C510054E06F6003020D46906686E0FF90635595
:100C6100E06F6003020D46C2199065787401F012BD
:100C710036AA751201020D4690668EE0600374017A
:100C8100F090667BE0FF906378E06F6003020D46B1
:100C910090667BE004F0E4F512906576F0020D4673
:100CA100301903020D46906345E07003020AC290B9
:100CB10062B4E06008906356741EF080069063563B
:100CC1007403F012354ED219E4F512906576F09066
:100CD100668704F0E490667AF0A3F02021677E0F26
:100CE1007FC0122807805E90668EE060037401F079
:100CF100301952906376E020E74B906378E0FF90E3
:100D0100667AE0FE6F600D906682E07007EE146F08
:100D11007033801390667AE004F0906332E0FFD381
:100D2100940440031234E29060007482F0A37401D1
:100D3100F0906378E0906002F07E607F007D0312A6
:100D41002F3B020AC2201903020E69E512706E12CE
:100D51003470EF60237E647F76906477E02404FD35
:100D6100122F3B906682E07009906356E0F5120203
:100D71000AC2E4F512020AC2906687E0D3943C40AD
:100D81003C906682E070369062B4E0703090668785
:100D910004F0122B91E4906476F0A37412F0906643
:100DA1007BE0906478F0A374FDF090610563A2018B
:100DB10090647A63A2017F12121B59809812369FA8
:100DC1008F26E526B401159060007483F0E4A3F04A
:100DD1007E607F007D02122F3B020AC2E526D3947A
:100DE10001401C9060007483F0A37401F0E5262497
:100DF100FEA3F07E607F007D03122F3B020AC2E555
:100E01001264016003020AC2906576E004F02021B9
:100E1100077E0F7FCA122807906576E0FFD3940101
:100E2100400B906356E0941E5003E004F0EFC3942E
:100E310005400DC219E4906578F01236AA020AC283
:100E41007C667D8390634AE0FAA3E0FB7F02123067
:100E5100CC7E647F76906477E02404FD122F3B9072
:100E61006356E0F512020AC2E51264016003020A48
:100E7100C2906578E014604624FE6042147003025B
:100E81000F5C24046003020AC2E4F51420251390C8
:100E910065787404F0906576E05401F075120102F2
:100EA1000AC29080027410F0E4906578F090657643
:100EB10004F075121290668374FFF0020AC2906604
:100EC10083E07003020F469064767480F09064783A
:100ED1007401F0E4A3F0A304F0A37430F0A3747BD5
:100EE100F0E4F526747D2526F582E43464F58374F7
:100EF1007DF0747E2526F582E43464F583E4F0E523
:100F0100262407906477F07C667D8390634AE0FA3B
:100F1100A3E0FB7F021230CC7E647F76E5262409B4
:100F2100FD122F3B906682E0601B12354ED219E410
:100F3100F512906576F090668704F0E490667AF099
:100F4100A3F0020AC2302507E4906578F08006908C
:100F510065787404F0751212020AC290800274104E
:100F6100F0751203906576E06401FFF09065787486
:100F710001F0EF7019906352E06013FCA3E0FDA350
:100F8100E0FEA3E0FF9066831218FA020AC29063A2
:100F91004EE0FCA3E0FDA3E0FEA3E0FF9066831218
:070FA10018FA020AC280FEEB
:010FA8002226
:10003600906377E0B444047F0180027F009063768A
:10004600E0B447047E0180027E00EE5F604A906362
:100056003FE0906378F0906340E0906379F09063BE
:1000660041E090637AF0906342E090637BF09063A6
:1000760043E090637CF0906344E090637DF090638E
:10008600777452F09062AE63A2019080A863A201D9
:100096007F06121B59020917906332E0C394085079
:1000A6000302092090633FE0FF906378E06F6003EE
:1000B600020920906340E0FF906379E06F600302DD
:1000C6000920906341E0FF90637AE06F60030209C4
:1000D60020906342E0FF90637BE06F60030209209B
:1000E600906343E0FF90637CE06F60030209209019
:1000F6006344E0FF90637DE06F6003020920906334
:1001060077E06444701A9080A8E0B4FF139062AE62
:1001160063A2019080A863A2017F06121B5980107A
:100126009062B2E09080ACF09062B3E09080ADF067
:1001360090668EE060037401F090668F7464F090B0
:1001460063777452F0906376E0646D60030202BADE
:100156007BFF7A0F79D51215137BFF7A0F79EF9013
:10016600633FE0F52FA3E0F530A3E0F531A3E0F51A
:1001760032A3E0F533A3E0F534121513752FFF759E
:10018600301075314C7532FF7533107534587BFF5E
:100196007A1079251215137BFF7A107961121513DF
:1001A6007BFF7A1079C71215137BFF7A1079F490CA
:1001B6006345E0F52FA3E0F530A3E0F531A3E0F5C4
:1001C600321215137BFF7A11791E90634EE0F52FDC
:1001D600A3E0F530A3E0F531A3E0F5321215137B69
:1001E600FF7A11794C906352E0F52FA3E0F530A326
:1001F600E0F531A3E0F5321215137BFF7A11797A17
:1002060090633BE0F52FA3E0F530A3E0F531A3E0E2
:10021600F5321215137BFF7A11799D906337E0F55D
:100226002FA3E0F530A3E0F531A3E0F53212151364
:100236007BFF7A1179BA1215137BFF7A1179E3A243
:1002460025E433F52F1215137BFF7A127913906686
:1002560082E0F52F1215137BFF7A12793E90668E97
:10026600E0F52F1215137BFF7A1279719062B4E0D4
:10027600F52F1215137BFF7A1279A3A217E433F533
:100286002F1215137BFF7A1279CF90667CE0F52F3B
:10029600A3E0F530A3E0F531A3E0F532A3E0F533B2
:1002A600A3E0F534121513122CF67BFF7A13791A94
:1002B60012151322906376E0644C70737E137F20D0
:1002C600FBFDFC1225FC90637EE0F527A3E0F528F4
:1002D600E4F52AE527906380F0A3E528F07E137FF6
:1002E6005B7C637D807B021225FCE4F529852882F0
:1002F600852783E0FF74802529F582E43463F5833E
:10030600EFF00528E528700205270529E529B41030
:10031600DC7E137F5E7C637D807B101225FC052AC4
:10032600E52AC3941040AC7E137F61122807229001
:100336006376E0646C7060F52B7E137F63FBFDFCD7
:100346001225FCE4F52AE4906380F0A3E52BF07E09
:10035600137F5B7C637D807B021225FCE4F529A874
:100366002BE6FF74802529F582E43463F583EFF0EC
:10037600052B0529E529B410E67E137F5E7C637D97
:10038600807B101225FC052AE52AC3940840B77E17
:10039600137F6112280722906376E0644B7061F543
:1003A6002974682529F582E43463F583E0603274A4
:1003B600682529F582E43463F583E0F460237468E4
:1003C6002529F582E43463F583E0FF747E2529F55B
:1003D60082E43463F583E0B507100529E529B408FE
:1003E600C09061047432F00209179063767421F0AC
:1003F6003021030209177E137F9E12280702091770
:10040600906376E0B4521A2021077E137FA6122845
:10041600079063767472F07E637F767D08122EB441
:1004260022906376E0644970452021077E137FB1F0
:1004360012280790637EE0F527A3E0F528E4F52966
:10044600852882852783E0FF74802529F582E43498
:1004560063F583EFF00528E528700205270529E5F1
:1004660029B480DC7E637F767D8A122EB422906367
:1004760076E0644370462021077E137FB912280771
:1004860090637EE0F527A3E0F528E4F52985288228
:10049600852783E493FF74802529F582E43463F588
:1004A60083EFF00528E528700205270529E529B41C
:1004B60080DB7E637F767D8A122EB422906376E09F
:1004C600645A70532021077E137FC2122807906357
:1004D6007EE0F527A3E0F5287C637D807B80AF284E
:1004E600AE2712351AE4F529852882852783E493F9
:1004F600FF74802529F582E43463F583EFF005283F
:10050600E528700205270529E529B480DB7E637F8F
:10051600767D8A122EB422906376E06444600302EC
:1005260005AE90637EE0FF64447003020917EFB4E2
:10053600310CC2217E137FCE122807020917906361
:100546007EE0B4300CD2217E137FDA12280702092E
:100556001790637EE0B4320CD2227E137FE7122816
:100566000702091790637EE0B4330CC2227E137F24
:10057600F512280702091790637EE0B4340CD223E3
:100586007E147F0412280702091790637EE0B435B3
:100596000CC2237E147F1112280702091790637E6E
:1005A600E0FF12001E020917906104E0701320217B
:1005B600077E147F1F1228079063767421F00209C4
:1005C600179061047432F0906376E0FFB45104C270
:1005D600AF80FEEF645770452021077E147F2D12F1
:1005E600280790637FE0906332F0E4F52990633248
:1005F600E0FFE529C39F400302091774802529F50A
:1006060082E43463F583E0FF90637EE0252924AD20
:10061600F582E43461F583EFF0052980D0906376A6
:10062600E0645360030206D12021077E147F38124E
:10063600280790633FE0FF9061B6E06F703C9063DF
:1006460040E0FF9061B7E06F7030906341E0FF904B
:1006560061B8E0B50724906342E0FF9061B9E0B568
:100666000718906343E0FF9061BAE0B5070C90630A
:1006760044E0FF9061BBE06F60169063767421F0F2
:100686003021030209177E147F4712280702091733
:10069600E4F529E4F515AF29FE74AD2529F582E4C4
:1006A6003461F583E0FD12357F0529E529C394FE03
:1006B60040E1C2AFE4907FF0F0A3F0907FFD74AA12
:1006C600F0A374FFF0A37455F080FE906376E064A7
:1006D6004F705A90637EE0F527A3E0F528E528459C
:1006E60027700A2021077E147F5012280720210731
:1006F6007E147F57122807E4F52974802529F58290
:10070600E43463F583E0852882852783F00528E5B0
:1007160028700205270529E529B480DE90668DE05C
:100726002480F090668CE03400F00209179063761E
:10073600E06445707490637EE0FEA3E0FF907FF076
:10074600EEF0A3EFF0D39400EE94044038907FF0DF
:10075600E0FEA3E0FF90668CE0FCA3E0FD9FEC9E2C
:100766004023E42FFFEE3401FED3ED9FEC9E50159F
:10077600C2AF907FFD74AAF0A374FFF0A37455F086
:10078600E4F5A780FE7E147F591228077BFF7A14B2
:100796007961907FF0E0F52FA3E0F53090668CE06C
:1007A600F531A3E0F532121513906376E0646560C7
:1007B6000302092090637EE0FFA3E0907FF0CFF074
:1007C600A3EFF0E4F527F528D3907FF1E095289084
:1007D6007FF0E095274020E4F5152528FFE527342E
:1007E60001FE852882852783E0FD12357F0528E5F1
:1007F600287002052780D17E147F6C122FC2EF4E1F
:100806006020120003906345EFF0120003906346E8
:10081600EFF0120003906347EFF012000390634875
:10082600EFF07E147F72122FC2EF4E60201200038B
:1008360090634EEFF012000390634FEFF012000347
:10084600906350EFF0120003906351EFF07E147F37
:1008560078122FC2EF4E6020120003906352EFF021
:10086600120003906353EFF0120003906354EFF00D
:10087600120003906355EFF07E147F7E122FC2EFB5
:100886004E602012000390633BEFF012000390636A
:100896003CEFF012000390633DEFF012000390630B
:1008A6003EEFF07E147F84122FC2EF4E60201200BE
:1008B60003906337EFF0120003906338EFF01200F5
:1008C60003906339EFF012000390633AEFF0E4F51A
:1008D60029E4F515E5292401FFE433FE74372529BB
:1008E600F582E43463F583E0FD12357F0529E529B9
:1008F600C3944340DCC2AFE4907FF0F0A3F0907F56
:10090600FD74AAF0A374FFF0A37455F0E4F5A78074
:0A091600FE7E637F767D08122EB48A
:0109200022B4
:1034AA00AE07EEC39430400BEED394395005EE24A8
:1034BA00D0FF22EEC39461400BEED394665005EE22
:1034CA0024A9FF22EEC39441400BEED39446500543
:0834DA00EE24C9FF22AF062217
:103641009062ADE004F070069062ACE004F090622C
:0A365100ACE0FEA3E0FF1235EB220F
:100003001236411234AAEFC454F0FEC00612364130
:080013001234AAD0E02FFF22F5
:10331400E4906983F0123641906984EFF0C39430ED
:103324004018E0FFD394395011906983E02405F5E7
:1033340082E43461F583EFF08011906983E0240521
:10334400F582E43461F583E4F0800C906983E00451
:10335400F0E0D3940840BE752A00752B00752C004C
:0C336400E4F52D7B017A617905121C67ED
:01337000223A
:042FC2008E2C8F2D95
:102FC6009062ACE4F0A374FFF0123641EF606EF449
:102FD600606B852D82852C83E493B507EC752E01F5
:102FE600E52D252EF582E4352CF583E493602590B6
:102FF60062ADE0252EFF9062ACE03400FE1235EBA8
:10300600E52D252EF582E4352CF583E493B50704EA
:10301600052E80CCE52D252EF582E4352CF583E4AE
:103026009370A6E52E24FFFFE434FFFE9062ADE028
:103036002FF09062ACE03EF07E007F0122E4FEFFBE
:013046002267
:1028EF007E147F8A122FC2EF4E70037F01227E1457
:1028FF007F8D122FC2EF4E600C123641EF24D02481
:10290F00FF92258002D2257E147F93122FC2EF4EA5
:10291F00600C123641EF24D0906682F08005E4906F
:10292F006682F07E147F99122FC2EF4E600C123622
:10293F0041EF24D090668EF08005E490668EF07E95
:10294F00147F9F122FC2EF4E600C123641EF24D02E
:10295F0024FF92178002C2177E147FA5122FC2EF99
:10296F004E600C123641EF24D09062B4F08005E433
:10297F009062B4F090633F63A20190667C63A20102
:10298F007F06121B5930173B7E147FAB122FC2EFFD
:10299F004E603012000390667CEFF01200039066D9
:1029AF007DEFF012000390667EEFF0120003906649
:1029BF007FEFF0120003906680EFF0120003906635
:0629CF0081EFF07F002201
:10342700906577E0C3947C40027F0A906577E0FE61
:1034370004F074B52EF582E43462F583EFF0BF0A29
:1034470027906577E0FF04F074B52FF582E43462C6
:10345700F583E4F0906577E0FF1230479065777465
:0934670008F09062B6E004F022C6
:1033CD009080007480F090633763A201F583F582DD
:1033DD0063A2017F08121B5990633F63A201908085
:1033ED008863A2017F0A121B599080927407F0A383
:1033FD0074D0F0A37406F0906349E0FF9080B1F0B3
:10340D009080E1EFF09080957455F0A3F0908000DE
:0A341D007401F090800974F0F022B1
:10324800908009E04410F09080A0E070609080A128
:103258007482F09080A874FFF0A3F0A3F0A3F07F2D
:10326800039080AEEFF0A374CBF09080007402F06E
:1032780090697312190600000000906973E090804D
:1032880040F0906974E0908041F0906975E090801A
:1032980042F0906976E0908043F0A3E4F0A3F0A3B5
:0D32A800F0A3F0908018F0A3F0A3F0A3F0C5
:0132B50022F6
:10337100908009E04440F09080D17482F07F039006
:1033810080DEEFF0A374CCF09080027402F09069BB
:103391007712190600000000906977E0908058F0DC
:1033A100906978E0908059F0906979E090805AF0C6
:1033B10090697AE090805BF0A3E4F0A3F0A3F0A31E
:0B33C100F0908030F0A3F0A3F0A3F028
:0133CC0022DE
:1031CE00908009E04420F09080B8E0706C9080B957
:1031DE007482F07F039080C6EFF07FCDA3EFF07F77
:1031EE00039080C4EFF0A374CDF09080C074FFF014
:1031FE00A3F0A3F0A3F09080017402F090697B120B
:10320E0019060000000090697BE090804CF09069F8
:10321E007CE090804DF090697DE090804EF090695A
:10322E007EE090804FF0A3E4F0A3F0A3F0A3F09023
:09323E008024F0A3F0A3F0A3F03A
:013247002264
:1030CC008C278D28A907EAFDE975F018A424ACFF1C
:1030DC00E5F034808F82F583EDF0EBFDE975F018A7
:1030EC00A4FFAEF024ACFBEE34808B82F583A3ED11
:1030FC00F08528828C83E0FDEF24A8FFEE3480FE5F
:10310C008F82F583EDF08528828C83A3E08F828EED
:10311C0083A3F0852882852783A3A3E0FDE975F0BE
:10312C0018A424A8FFE5F03480FE8F82F583A3A3B6
:10313C00EDF08528828C83A3A3A3E08F828E83A3DA
:04314C00A3A3F02227
:062EB4008D2CAB07AA06FD
:102EBA00908000E030E5079065797401F02290690E
:102ECA0073E0FCA3E0FDA3E0FEA3E0F5308E2F8DB6
:102EDA002E8C2DAE02AF038E838F8263A201E52F63
:102EEA00540744C0F58385308263A201AF2C121BBC
:102EFA00CBE4FCFDFEE530252CF530EE352FF52F21
:102F0A00ED352EF52EEC352DF52D908040E52DF082
:102F1A00A3E52EF0A3E52FF0A3E530F0908000742E
:102F2A0020F0AF30AE2FAD2EAC2D9069731218FA87
:012F3A002274
:062F3B008D27AB07AA067A
:102F4100908002E030E5079065797403F022906982
:102F510077E0FCA3E0FDA3E0FEA3E0F52B8E2A8D34
:102F6100298C28AE02AF038E838F8263A201E52AEA
:102F7100540744D0F583852B8263A201AF27121B2E
:102F8100CBE4FCFDFEE52B2527F52BEE352AF52AB2
:102F9100ED3529F529EC3528F528908058E528F0FC
:102FA100A3E529F0A3E52AF0A3E52BF090800274B4
:102FB10020F0AF2BAE2AAD29AC289069771218FA10
:012FC10022ED
:022C46008F27D6
:102C4800908001E030E5099065797402F07F0022F8
:102C580090697BE0FCA3E0FDA3E0FEA3E0F52B8EEA
:102C68002A8D298C2890667C63A201E52A540744A2
:102C7800C8F583852B8263A2017F06121BE1E52B31
:102C88002406F52BE4352AF52AE43529F529E43517
:102C980028F52890657A63A201E52A540744C8F507
:102CA80083852B8263A201AF27121BE1E4FCFDFEA2
:102CB800E52B2527F52BEE352AF52AED3529F529BB
:102CC800EC3528F52890804CE528F0A3E529F0A3F9
:102CD800E52AF0A3E52BF09080017420F0AF2BAE2D
:0D2CE8002AAD29AC2890697B1218FAAF279D
:012CF50022BC
:102703009081E0E0F52705270527052705270527FD
:1027130005270527052705270527908010E0F52ABB
:10272300A3E0F52BA3E0F52CA3E0F52D9081E1E0E8
:10273300F527052705270527052705270527052746
:10274300052705270527908014E0F52EA3E0F52F34
:10275300A3E0F530A3E0F531E530B52C08E531B55C
:102763002D037F0022E4F527E530540744E0F58389
:1027730085318263A20190637663A2017F08121CF4
:102783001190637863A2019062AE63A2017F061287
:102793001B59906376E0F528A3E0F529E4F527902B
:1027A3006376E0702AA3E024F8F527E53054074464
:1027B300E0F58385318274082582F582E43583F55B
:1027C3008363A20190637663A201AF27121C11AE4B
:1027D30028E4FCFDE5312529F531E5303EF530ED02
:1027E300352FF52FEC352EF52E908014E52EF0A322
:1027F300E52FF0A3E530F0A3E531F09080007440BD
:03280300F0AF270C
:0128060022AF
:101E0B009081E6E0F52705270527052705270527F8
:101E1B0005270527052705270527908028E0F52AA4
:101E2B00A3E0F52BA3E0F52CA3E0F52D9081E7E0E3
:101E3B00F527052705270527052705270527052747
:101E4B0005270527052790802CE0F52EA3E0F52F1D
:101E5B00A3E0F530A3E0F531E4F527E530B52C0A26
:101E6B00E531B52D05C21E021F77E530540744F04E
:101E7B00F58385318263A20190637663A2017F08AB
:101E8B00121C11906376E0F528A3E0F529E52945AE
:101E9B002870099080027410F07F0022906683E016
:101EAB00FFF46030906378E06F6003021F3E906632
:101EBB0084E0FF906379E06F7079906685E0FF9026
:101ECB00637AE06F706D906686E0FF90637BE06FE6
:101EDB006031805F906378E0906683F0906379E087
:101EEB00906684F090637AE0906685F090637BE077
:101EFB00906686F090637CE0FFA3E090634ACFF09E
:101F0B00A3EFF0906376E0702AA3E024F8F527E5C1
:101F1B0030540744F0F58385318274082582F582AD
:101F2B00E43583F58363A20190637663A201AF2747
:101F3B00121C11AE28E4FCFDE5312529F531E53005
:101F4B003EF530ED352FF52FEC352EF52EAF2DAEB2
:101F5B002CAD2BAC2AAB31AA30A92FA82ED312183B
:101F6B00E940099080027410F07F002290802CE5EC
:101F7B002EF0A3E52FF0A3E530F0A3E531F0908030
:061F8B00027440F0AF27D4
:011F9100222D
:101F92009081E3E0F5270527052705270527052773
:101FA2000527052705270527052790801CE0F52A28
:101FB200A3E0F52BA3E0F52CA3E0F52D9081E4E05E
:101FC200F5270527052705270527052705270527BF
:101FD200052705270527908020E0F52EA3E0F52FA1
:101FE200A3E0F530A3E0F531E4F527E530B52C0A9E
:101FF200E531B52D05C21F0220E8E530540744E85B
:10200200F58385318263A20190600463A2017F0E91
:10201200121C27906004E0F528A3E0F52990600CDB
:10202200E0FFF4604A90667CE0FEEF6E7079A3E018
:10203200FF90600DE06F706F90667EE0FF90600E23
:10204200E06F706390667FE0FF90600FE06F705703
:10205200906680E0FF906010E06F704B906681E0C8
:10206200FF906011E06F703FE4906013F080089081
:10207200601374FFF0D2D9906004E0702AA3E024C8
:10208200F2F527E530540744E8F583853182740E72
:102092002582F582E43583F58363A20190600463AF
:1020A200A201AF27121C27AE28E4FCFDE531252949
:1020B200F531E5303EF530ED352FF52FEC352EF5C7
:1020C2002EAF2DAE2CAD2BAC2AAB31AA30A92FA846
:1020D2002ED31218E95006E529452870099080018F
:1020E2007410F07F0022908020E52EF0A3E52FF0FF
:1020F200A3E530F0A3E531F09080017440F0AF2702
:0121020022BA
:042807008E2C8F2D57
:10280B00908000E030E5079065797401F0229069C3
:10281B0073E0FCA3E0FDA3E0FEA3E0F5338E328D65
:10282B00318C30E533FFE5325407FEE42FF52FEE04
:10283B0034C0F52E852F82F5837423F0052FE52FF9
:10284B007002052E532EC7F582852E83740AF00570
:10285B002FE52F7002052E532EC790633F63A20105
:10286B00852E83852F8263A2017F06121BCB7406F4
:10287B00252FF52FE4352EF52E852C83852D8263A0
:10288B00A201852E83852F8263A201121BAFE4FC6C
:10289B00FDFE906973E0F8A3E0F9A3E0FAA3E02F43
:1028AB00FFEE3AFEED39FDEC38FCEF2408FFE43E79
:1028BB00FEE43DFDE43CFC9069731218FA906973D9
:1028CB00E0908040F0906974E0908041F0906975E1
:1028DB00E0908042F0906976E0908043F090800029
:0328EB007420F066
:0128EE0022C7
:0A25FC008E2C8F2D8C2E8D2F8B302E
:10260600908000E030E5079065797401F0229069CA
:1026160073E0FCA3E0FDA3E0FEA3E0F5368E358D66
:10262600348C33E536FFE5355407FEE42FF532EEFC
:1026360034C0F531853282F5837423F00532E532F4
:10264600700205315331C7F582853183740AF0056E
:1026560032E532700205315331C790633F63A20100
:1026660085318385328263A2017F06121BCB7406F5
:102676002532F532E43531F531852C83852D82639B
:10268600A20185318385328263A201121BAF8F3787
:10269600EF2532F532E43531F531E5306017852E18
:1026A60083852F8263A20185318385328263A201ED
:1026B600AF30121BCBE53724082530F530FFE4FC9C
:1026C600FDFEE5362FF536EE3535F535ED3534F5C7
:1026D60034EC3533F533908040E533F0A3E534F040
:1026E600A3E535F0A3E536F09080007420F0AF3610
:0C26F600AE35AD34AC339069731218FAA5
:0127020022B4
:062AB6008E278F288D29F8
:102ABC00908000E030E5079065797401F022906910
:102ACC0073E0FCA3E0FDA3E0FEA3E0F52F8E2E8DBA
:102ADC002D8C2CE52FFFE52E5407FEE42FF52BEE65
:102AEC0034C0F52A852B82F5837423F0052BE52B56
:102AFC007002052A532AC7F582852A83EBF0052B31
:102B0C00E52B7002052A532AC790633F63A2018507
:102B1C002A83852B8263A2017F06121BCB740625A8
:102B2C002BF52BE4352AF52A85278385288263A289
:102B3C0001852A83852B8263A201AF29121BCB74DA
:102B4C00082529F529FFE4FCFDFEE52F2FF52FEED6
:102B5C00352EF52EED352DF52DEC352CF52C9080F4
:102B6C0040E52CF0A3E52DF0A3E52EF0A3E52FF026
:102B7C009080007420F0AF2FAE2EAD2DAC2C906950
:042B8C00731218FAAE
:012B90002222
:023047008F40B8
:10304900908000E030E5079065797401F02290697D
:1030590073E0FCA3E0FDA3E0FEA3E0F5448E438DFD
:10306900428C41E544FFE5435407FEE42FFFEE346B
:10307900C09062B563A201F5838F8263A201AF405C
:10308900121BCBE4FCFDFEE5442540F544EE354337
:10309900F543ED3542F542EC3541F541908040E587
:1030A90041F0A3E542F0A3E543F0A3E544F09080A5
:1030B900007420F0AF44AE43AD42AC419069731245
:0230C90018FAF3
:0130CB0022E2
:0629D5008E278F28AB05E0
:1029DB00908000E030E5079065797401F0229069F2
:1029EB0073E0FCA3E0FDA3E0FEA3E0F52E8E2D8D9E
:1029FB002C8C2BE52EFFE52D5407FEE42FF52AEE4C
:102A0B0034C0F529852A82F5837423F0052AE52A3B
:102A1B00700205295329C7F582852983EBF0052A16
:102A2B00E52A7002052990633F63A20185298385FE
:102A3B002A8263A2017F06121BCB7406252AF52A74
:102A4B00E43529F5295329C7E527852A828529836A
:102A5B00F0052AE52A700205295329C7F582852935
:102A6B0083E528F0052AE52A700205295329C7E5D5
:102A7B002E240AF52EE4352DF52DE4352CF52CE41A
:102A8B00352BF52B908040E52BF0A3E52CF0A3E53F
:102A9B002DF0A3E52EF09080007420F0AF2EAE2D1C
:0A2AAB00AD2CAC2B9069731218FAE1
:012AB50022FE
:0A369400E4FEEEC39F50030E80F821
:01369E002209
:1035EB00A2AF9226C2AF438E2075D2028F828E83FA
:0C35FB00E0FFE4F5D2538EDFA22692AF71
:0136070022A0
:10357F00E5D220E0FBA2AF9226C2AF43D2028F82E8
:10358F008E83EDF075D25063D250A22692AFE5D262
:03359F0020E0FB2E
:0135A2002206
:10315000E4FDED2401FFE433FE1235EB74372DF569
:1031600082E43463F583EFF00DBD3FE6E4FDED242A
:103170007FFFE433FE1235EB742D2DF582E43461CC
:10318000F583EFF0742D2DF582E43461F583E07062
:103190001B742D2DF582E43461F5837420F0742EB8
:1031A0002DF582E43461F583E4F080040DBD80BE2A
:1031B000E49061ACF0FDEDFF7E001235EB74AD2DB7
:0D31C000F582E43461F583EFF00DBDFEE90A
:0131CD0022DF
:02351A008B2CF8
:10351C00A2AF9226C2AF85A22D53A2FE8E838F82BC
:10352C0005A28C838D827409121C55E52C53A2FEC6
:10353C0043A220121C5753A2DF852DA2A22692AFC4
:01354C00FF7F
:01354D00225B
:10360800A2AF9226C2AF8C838D82EF121C5543A2C3
:0C36180020121C5753A2DFA22692AFFF25
:013624002283
:0235A3008F2770
:1035A500A2AF9226C2AFE4F5838D827406121C5534
:1035B500E52743A220121C5753A2DFA22692AF7F14
:0135C5000104
:0135C60022E2
:0235C7008F274C
:1035C900A2AF9226C2AFE4F5838D82740A121C550C
:1035D900E52743A220121C5753A2DFA22692AF7FF0
:0135E90001E0
:0135EA0022BE
:101A7E00A907E7FFA805EF93C3966008403B74FCE7
:101A8E002FFF80F00F08EF93C3966008402B74FB76
:101A9E002FFF80E00F08EF93C3966008401B74FA87
:101AAE002FFF80D00F08EF93D3966008400B74F988
:101ABE002FFF80C01F1F1F1F1FEF54FEF80303F7D9
:101ACE00E893FC08E893FD08E893FE08E893FF22EC
:101ADE0009E993C39D6008402974FB29F980F10937
:101AEE00E993C39E6008401A74FA29F980E209E965
:101AFE0093D39F6008400B74F929F980D3191919F3
:101B0E001919E9C313C313FF22740093F8ECC39899
:101B1E004024701F740193F8EDC39840197014742B
:0E1B2E000293F8EEC398400E7009740393F80A
:101B3C00EFC39840037F00227F0122EDF8E6F00806
:101B4C00A3DFFA22EDF8E0F608A3DFFA22E0A363A4
:101B5C00A201F0A363A201DFF475A2002263A2012B
:101B6C00F0A363A20122E0A363A201F0A363A2018C
:101B7C00E0A363A201F0A363A201E463A201F0A3BA
:101B8C0063A201DFE175A20022E0A363A2016DFE56
:101B9C00936CFDEE058393FC158363A201DFEA755C
:101BAC00A200227F00E493A363A201F00F600CA3B8
:101BBC00E583C2E3F58363A20180EA75A20022E00B
:101BCC00A363A201F0A3E583C2E3F58363A201DF63
:101BDC00EE75A20022E0A363A201F0A3E583C2E4A8
:101BEC00D2E3F58363A201DFEC75A20022E0A363CC
:101BFC00A201F0A3E58344F8C2E5F58363A201DFFB
:101C0C00EC75A20022E583C2E3F583E0A363A20195
:101C1C00F0A363A201DFEE75A20022E583C2E4D239
:0A1C2C00E3F583E0A363A201F0A337
:101C360063A201DFEC75A20022E58344F8F583E098
:101C4600A363A201F0A363A201DFEE75A20022F94D
:101C560022C002C004C00612FFF0D006D004D00293
:011C6600225B
:10001E00BF360BD20DE4F546F547F562F563BF37F3
:04002E0002C20D22DB
:1032B600C2A943890290696EE0FFF58C8F8A75D9A1
:1032C6000475DA4875DB3175DC4975DD4975DE3123
:1032D600E4F5E9F5F9F5EBF5FB90696CE060167538
:1032E600EC1075ED10E4F5FCF5FD755E08755C10E7
:1032F600755D01801375EC8075ED80E4F5FCF5FDD8
:0E330600755E80F55C755D10E4F5EEF5FE2257
:0E368500E4FFD28C75D84075B740D2AED2AFFC
:013693002214
:0300330002226A3C
:0B226A00C0E0C083C082C0D075D00867
:10227500C2AF30DC56C3E5EC95EEC3955E5012E572
:102285005D25ECF5EC30D70405FC801685FCFC805B
:1022950011C3E5EC955DF5EC30D70415FC8003859D
:1022A500FCFC300D24854782854683E590F0054783
:1022B500E54770020546F582854683E5EEF005475C
:1022C500E5477002054653460FC2DC30D929300D6B
:1022D50024854782854683E590F00547E5477002EA
:1022E5000546F582854683E5EBF00547E54770022F
:1022F500054653460FC2D930DA51E55C700405FC3A
:102305008010E55C25ECF5EC30D70405FC800385F1
:10231500FCFC300E34E5485480F545E54825E0F5EC
:10232500483097020548200C03634801202F1A0501
:102335005FE55F54077012535F3FE55F1313135456
:102345001F244AF8A648754800C2DA30DB71E55CFF
:10235500700405FD8010E55C25EDF5ED30D704052D
:10236500FD800385FDFDE560655B6029E55B540740
:102375007013E55B131313541F2452F8E6F5492037
:1023850009036349FFE549339296E54925E0F54997
:10239500055B535B3FB292300D23854782854683AB
:1023A500E590F00547E54770020546F582854683C9
:1023B500E4F00547E5477002054653460FC2DBD2F8
:0123C500AF68
:0923C600D0D0D082D083D0E032E7
:1023CF000A20C2F5EEE4EDEEE920E1F3F4E5F020AA
:1023DF00EFE5F0E5EFEEEBEDE5ED2120003E2A2CE9
:1023EF00312CCFE0F0E0ECE5F2F0FB20F1E8EDF579
:1023FF00F0EEEDEDEEE3EE20EFEEF0F2E02E20CF7B
:10240F00EEF2EEEAEEE2FBE920F0E5E6E8EC0A0098
:10241F003E4C2C4230312C256C752CD1EAEEF0EE6F
:10242F00F1F2FC20EEE1ECE5EDE02C35302C313013
:10243F00302C3230302C3330302C3630302C31328F
:10244F0030302C323430302C343830300A003E42A9
:10245F002C4731302C2562752CC8EDE2E5F0F1E800
:10246F00FF20EDE020EFF0E8B8ECE50A003E422C4B
:10247F004731312C2562752CC8EDE2E5F0F1E8FF0C
:10248F0020EDE020EFE5F0E5E4E0F7E50A003E534C
:10249F002C4730342C2562752CCFF0E8B8ECEDFBCF
:1024AF00E920E1F3F4E5F02028E1E0E9F2290A0060
:1024BF003C21003C4230313D003C4731303D003C37
:1024CF004731313D003C4730343D000008040C02D9
:0B24DF000A060E0109050D030B070F94
:10362B005266900000000000000000000000000047
:05363B0000000000008A
:0100320022AB
:10347000301434E4906476F0A3E571F090667BE05C
:10348000906478F0A3E570F09067E763A201906420
:103490007A63A201AF71121B59C214E4F57175650C
:0A34A000677566E77F01227F0022B6
:10365B0090696D74FFF0A374B8F0E490696CF0900E
:0A366B006969F01224EA1232B62257
:10354E0075647EC207D20EC214C22FC211C201C24E
:10355E0012D200E4F571F572F55BF560F574F57550
:10356E007570097565677566E7C291C290123685EA
:01357E00222A
:1034E200EF24FCFF2572F572AE74906379E0F570FB
:1034F200E4FDEDC39F501C747A2DF582E43463F52C
:1035020083E0FC74672EF582E43468F583ECF00DF9
:073512000E80DF8E74D290E1
:01351900228F
:102B9100E4FF0F2405F582E43461F5837408F00F36
:102BA10074052401F582E43461F583E4F07C667DEB
:102BB10095FEED1DAA0470011CF5828A83E0FBAA33
:102BC100070F74052AF582E43461F583EBF00EBE3C
:102BD10004E07C667D99E4FEED1DAA0470011CF5FC
:102BE100828A83E0FBAA070F74052AF582E4346127
:102BF100F583EBF00EBE04E07C667D9DE4FEED1DE9
:102C0100AA0470011CF5828A83E0FBAA070F7405F0
:102C11002AF582E43461F583EBF00EBE04E07C66B4
:102C21007DA1E4FEED1DAA0470011CF5828A83E0FA
:102C3100FBAA070F74052AF582E43461F583EBF0F2
:042C41000EBE04E0DF
:012C4500226C
:10210300300D2DC3E5479563FFE5469562FED3EF9A
:102113009440EE940040197B087D40AF63AE621299
:102123002AB6E5632440FFE43562540FF5628F63FA
:10213300201905D291D290223013179066A4E06043
:1021430017301814C21814F0E0700D740AF0D2128C
:1021530080069066A47401F0E55F5438655A6059AF
:10216300E55A24085438F55A131313541F244AF814
:10217300E6F56C0566E566AE657002056514F582E5
:102183008E83E56CF0057130141EE571D3948040A5
:1021930024E4F571C2147565677566E77E237FCF06
:1021A300FBFDFC1225FC800D9066A3E0FFE571C3E7
:1021B3009F4002D214D291809FE560655B6053E536
:1021C3006024085438FFE55B54386F60047E018057
:1021D300027E00E57260047D0180027D00EE5D7089
:1021E3000302226974672575F582E43468F583E098
:1021F300FEE560131313541F2452F8A60605758FCA
:10220300601572E572D394055004D21380B1C213E2
:1022130080ADE572602674672575F582E43468F550
:1022230083E0FFE560131313541F2452F8A6070538
:1022330075E56024085438F56015722230902590B6
:10224300669EE0FCA3E0FDA3E0FEA3E0FFE4FAF951
:10225300F8EF2401FFEA3EFEE93DFDE83CFC906611
:072263009E1218FAC290223E
:0B369F00301205C2127F01227F0022C2
:102CF6007BFF7A2379EC12151390696CE06033A39D
:102D0600E0FEA3E0FFC3E49FFFE49EFEAB07FA33B9
:102D160095E0F9F87F007EC27D017C001218498F8C
:102D2600328E318D308C2F7BFF7A24791F1215134A
:102D3600803290696DE0FEA3E0FFC3E49FFFE49E4E
:102D4600FEAB07FA3395E0F9F8E47F207E1CFDFC24
:102D56001218498F328E318D308C2F7BFF7A247971
:102D66001F1215137BFF7A24795DA20CE433F52F2D
:102D76001215137BFF7A24797CA209E433F52F120E
:102D860015137BFF7A24799D9066A3E0F52F121523
:022D9600132206
:1024EA007E247FBF122FC2EF4E70037F01227E240B
:1024FA007FC2122FC2EF4E7003022591123314903D
:10250A00697F1218FAE4FFFEFDFC90697FE0F8A3E8
:10251A00E0F9A3E0FAA3E0FBC31218E96025906989
:10252A007FE0F8A3E0A3E0A3E0E47F207E1CFDFCAB
:10253A001218491218DB90696DEEF0A3EFF0E490DF
:10254A00696CF0E47FB07E04FDFC90697FE0F8A33B
:10255A00E0F9A3E0FAA3E0FBD31218E94038906946
:10256A006C7401F090697FE0F8A3E0A3E0A3E07F38
:10257A00007EC27D017C001218491218DB90696D39
:10258A00EEF0A3EFF0800F90696D74FFF0A374B8BA
:10259A00F0E490696CF07E247FC8122FC2EF4E607F
:1025AA000C123641EF24D024FF920C8002C20C7E1A
:1025BA00247FCE122FC2EF4E600C123641EF24D088
:1025CA0024FF92098002C2097E247FD4122FC2EF0F
:1025DA004E600A1233149066A3EFF080069066A349
:1025EA00740AF09066A3E0D3942740037427F07F1F
:0125FA0000E0
:0125FB0022BD
:0336AA00C2AE228B
:102E3400020921E493A3F8E493A34003F68001F28A
:102E440008DFF48029E493A3F85407240CC8C3339F
:102E5400C4540F4420C8834004F456800146F6DF6E
:102E6400E4800B0102040810204080903625E47EA3
:102E7400019360BCA3FF543F30E509541FFEE49363
:102E8400A360010ECF54C025E060A840B8E493A32A
:102E9400FAE493A3F8E493A3C8C582C8CAC583CA55
:102EA400F0A3C8C582C8CAC583CADFE9DEE780BE0D
:013640000089
:10180D0075F008758200EF2FFFEE33FECD33CDCC92
:10181D0033CCC58233C5829BED9AEC99E582984015
:10182D000CF582EE9BFEED9AFDEC99FC0FD5F0D6F2
:10183D00E4CEFBE4CDFAE4CCF9A88222B800C1B91C
:10184D000059BA002DEC8BF084CFCECDFCE5F0CB5A
:10185D00F97818EF2FFFEE33FEED33FDEC33FCEB93
:10186D0033FB10D703994004EB99FB0FD8E5E4F94E
:10187D00FA227818EF2FFFEE33FEED33FDEC33FC3B
:10188D00C933C910D7059BE99A4007EC9BFCE99A2F
:10189D00F90FD8E0E4C9FAE4CCFB2275F010EF2F74
:1018AD00FFEE33FEED33FDCC33CCC833C810D70774
:1018BD009BEC9AE899400AED9BFDEC9AFCE899F8AF
:0E18CD000FD5F0DAE4CDFBE4CCFAE4C8F92242
:0E18DB00C3E49FFFE49EFEE49DFDE49CFC221E
:1018E900EB9FF5F0EA9E42F0E99D42F0E89C45F055
:0118F90022CC
:0C18FA00ECF0A3EDF0A3EEF0A3EFF02261
:10190600A8828583F0D083D08212191D12191D1268
:10191600191D12191DE473E493A3C583C5F0C5838D
:10192600C8C582C8F0A3C583C5F0C583C8C582C82B
:01193600228E
:1014B100E53B242FF8E6053B22782C302D02782FCE
:1014C100E475F0011219DE0219372026EB7F2ED2C6
:1014D100268018EF540F2490D43440D4FF302A0BC7
:1014E100EF24BFB41A0050032461FFE53C600215EC
:1014F1003C053FE53F7002053E302D0D782CE4752B
:10150100F0011219DEEF02197D0234277403D22D86
:101511008003E4C22DF53B8B2C8A2D892EE4F53C0A
:10152100F53EF53FE53C60077F201214EC80F57530
:101531003DFFC227C226C228C229C22BC22CC22EFD
:101541001214BAFF700D302D057F001214FDAF3F4C
:10155100AE3E22B4255FC2D5C22A1214BAFF24D0EE
:10156100B40A00501A75F00A783C30D50508B6FF68
:101571000106C6A426F620D5047002D22980D924FA
:10158100CFB41A00EF5004C2E5D22A0216FDD227C9
:1015910080C6D22680C0D22880BCD2D580BAD22BB8
:1015A10080B47F201214EC2028077401B53C004060
:1015B100F11214B1FF1214EC021525D22ED22C8097
:1015C100951214B1FB1214B1FA1214B1F94A4B700D
:1015D1000679CE7A177BFF20282EE53C602A7E0013
:1015E1008E8275830012195060060EEE653D70F013
:1015F100C2D5EBC0E0EAC0E0E9C0E0EE121744D08A
:10160100E0F9D0E0FAD0E0FB121937FF60AAEBC095
:10161100E0EAC0E0E9C0E01214ECD0E02401F9D026
:10162100E03400FAD0E0FBE53D0460DCD53DD98033
:10163100877BFF7A177940D228809C7910800279C4
:1016410008C22CC22E8008D2D5790A8004790AC238
:10165100D5E53D047002F53DE4FAFDFEFF1214B13B
:10166100FC7B082027131214B1FD7B1030260A12CF
:1016710014B1FE1214B1FF7B20EC3382D592D55008
:1016810013C3E43026069FFFE49EFEE42027039D5A
:10169100FDE49CFCE4CBF8C227EC700CCFCECDCCA2
:1016A100E824F8F870F38017C3EF33FFEE33FEED53
:1016B10033FDEC33FCEB33FB994002FB0FD8E9EB34
:1016C100302705F8D0E0C448B227C0E00AEC4D4EFF
:1016D1004F78207B0070C2EAB53D0040BCC0E012EB
:1016E1001746D0F0D0E0202704C4C0E0C4B227C020
:1016F100F01214D5D0F0D5F0EB021525121A3D15D4
:10170100C253163C5815934C158F4216404F16483C
:0F1711004416484915A843164E5516324616324F
:101720004516324717EE5015972D159B2E15BE2BDB
:10173000159F2315BC2017D72A155748000015B64A
:101740003F3F3F00790AA2D5202914302B09B91058
:10175000020404B9080104A2D5202C02500104207F
:1017600028689228B53C005034C0E07F2030291909
:101770007F30A228722C722B500F12179DC228C2E4
:101780002CC22BC22E7F30800F302B03E9C0E01219
:1017900014EC302B03D0E0F9D0E0B53CCC302B1763
:1017A0007F30B9100C1214EC7F58302A077F7880F4
:1017B00003B908031214EC3028057F2D0214EC7FC6
:1017C00020202EF87F2B202CF322922880CF286E09
:1017D000756C6C2900D2271214B13027F8C2277813
:1017E0003C30D50108F60215572D504349581214C4
:1017F000B12403B405004001E49017E9931214DD0D
:0D180000743A1214DDD229753C0402163C26
:101C67008B278A288929E4F533F532F531F530F5E4
:101C77002EF52FE52B452C452A6012EBC0E0EAC074
:101C8700E0E9C0E0AB2AAA2BA92C1219EEAB270575
:101C970029E529AA287002052814F9121937F534FD
:101CA700C394094007E534D3940D40E1E53464203B
:101CB70060DBE534B42D05432F038016E534B42BE0
:101CC70005432F01800C74FF2529F52974FF35285A
:101CD700F528E52D60046410703FAB27AA28A929D1
:101CE70012193764306009E52D702E752D0A802989
:101CF700900001121950FF64786004EFB458134341
:101D07002F01752D1074022529F529E43528F528AA
:101D17008007E52D7003752D08AB270529E529AA4E
:101D2700287002052814F9121937F534C394614055
:101D37000AE534D3947A50035334DF74D02534F54D
:101D470034C3940A400CE5349411406D74F925347A
:101D5700F534E534D3952D5060432F01853338850D
:101D67003237853136853035AF2D7E00E4FCFDAB4B
:101D770033AA32A931A83012198FC8ECC8C9EDC9E6
:101D8700CAEECACBEFCBE4FCFDFEEB2534F533EE10
:101D97003AF532ED39F531EC38F530AF33AE32ADD7
:101DA70031FCAB38AA37A936A835D31218E9500346
:101DB700021D20432F04021D20E52F20E003E480AD
:101DC7002DE52B452C452A601EAB27E52924FFF975
:101DD700E52834FFFAEBC0E0EAC0E0E9C0E0AB2A4F
:101DE700AA2BA92C1219EEE52F30E20774FFFFFE8C
:101DF700FDFC22E52FAF33AE32AD31AC3030E1031D
:041E07000218DB22C0
:10193700BB010689828A83E0225002E722BBFE02AE
:09194700E32289828A83E49322E1
:10195000BB010CE58229F582E5833AF583E022504C
:1019600006E92582F8E622BBFE06E92582F8E22296
:0D197000E58229F582E5833AF583E49322B0
:10197D00BB010689828A83F0225002F722BBFE0149
:02198D00F32243
:10198F00E88FF0A4CC8BF0A42CFCE98EF0A42CFCF7
:10199F008AF0EDA42CFCEA8EF0A4CDA8F08BF0A475
:1019AF002DCC3825F0FDE98FF0A42CCD35F0FCEBD4
:1019BF008EF0A4FEA9F0EB8FF0A4CFC5F02ECD3999
:0F19CF00FEE43CFCEAA42DCE35F0FDE43CFC2206
:1019DE00FAE6FB0808E6F925F0F618E6CA3AF6220A
:1019EE00BB011A89828A83D0F0D0E0F8D0E0F9D01A
:1019FE00E0FAD0E0FBE8C0E0C0F0021A6C5016E945
:101A0E00F8D083D082D0E0F9D0E0FAD0E0FBC082EB
:101A1E00C083021A63BBFE16E9F8D083D082D0E0F1
:0F1A2E00F9D0E0FAD0E0FBC082C083021A752223
:101A3D00D083D082F8E4937012740193700DA3A338
:101A4D0093F8740193F5828883E47374029368604C
:061A5D00EFA3A3A380DF4C
:091A6300EBF608EAF608E9F622A8
:091A6C00EBF0A3EAF0A3E9F0227B
:091A7500EBF208EAF208E9F222A2
:00000001FF
